:1000000018308A0000280000491943104529D227DA
:1000100052002010CD2AD4222000AB183217300015
:10002000AB1830173500A01539173000A015371759
:100030003500A01536173000A01534173500A0156F
:1000400033173000A015311735002010301730005D
:10005000A01631173500A01633173000A01634173C
:100060003500A01636173000A01637173500A01639
:1000700039173000AD1830173500202A4F274510AA
:10008000432754262E104F234600CD1264105429C6
:100090004521CC22A029452A201020002010201024
:1000A0000001CD126410C220D3292010A029452AB6
:1000B00020102000201020100001CD1264105439AF
:1000C0006531EC32A0316F39EE3272002010201011
:1000D00020100001A01A6B247A00A01B6B247A0068
:1000E00031186B247A00B11A6B247A00CD12641097
:1000F000C230F339A0316F39EE3272002010201077
:100100002010000120103518483D0001A0183018BB
:10011000483D000120193018483D000120193518CC
:10012000483D0000CD126410C230F339A03661376B
:10013000E13365002010C434F330623665320001CB
:1001400020102010201C3010483D000120102010ED
:1001500031193010483D000120102010311B3010A3
:10016000483D00012010201032183010483D000199
:1001700020102010321A3010483D000120102010AD
:10018000321C3010483D000120102010331930106F
:10019000483D000020182E1800012D18AE1A00014D
:1001A000AD182E180001AD18AE1A00012D192E1829
:1001B00000012D19AE1A0001AD192E180001AD195C
:1001C000AE1A00012D1A2E1800012D1AAE1A0001C8
:1001D000AD1A2E180001AD1AAE1A00012D1B2E18F3
:1001E00000012D1BAE1A0001AD1B2E180001AD1B26
:1001F000AE1A0001CD126410B23BE13C202C6F3BE3
:10020000653920002010C434F330623665320001B5
:10021000201045376131EC3264100000CD126410BB
:10022000D837F63272106639E5382E0020102010CB
:10023000000120103217B035483D00012010321760
:10024000B235483D000120103217B435483D000159
:1002500020103217B635483D000120103217B8354E
:10026000483D000120103317B035483D00012010F3
:100270003317B235483D000120103317B435483DDF
:100280000000CD126410CC377728E1397310D332D7
:10029000EE3900012010201020100000CD12641053
:1002A000C8346734D030F339A02965377300201083
:1002B000201020004927BA204E26200049273A2244
:1002C000472A2000CD126410CF3A7438753AA02620
:1002D0006F326500B2316810C63A6C362021F234B4
:1002E000E43365100001B23168104826C615D33AD0
:1002F0006210C63A6C360001A018633420286139B8
:100300006110C63A6C3620100000CD126410D23451
:1003100067347410CD3478002029E933683AA0316D
:10032000681700012014CC15D2142F1920100001D9
:100330002014D215CC142F1920100001202665336B
:100340007410A03168170000CD126410CC32663AE8
:100350002010CD347800202665337410A031681742
:1003600000012014D215CC142F19201000012014E4
:10037000CC15D2142F19201000012029E933683A36
:10038000A03168170000CD126410D33A6210F6371E
:10039000EC3AED3200012010201020100000CD12A8
:1003A0006410D0214D10C637F236613A0001202684
:1003B0004A10A02A7010F43720193421693A00013C
:1003C000A024B229A02A7010F43720193421693AE8
:1003D00000012029E933683A2D2520102019342105
:1003E000693A00012029E933683A2D2520102019A7
:1003F0003021693A00012029E933683A2D2520107F
:10040000A0183821693A00012029E933683A2D25DE
:100410002010A0183621693A00002028411A351909
:100420003510C416C1367010F61800012023753639
:100430006C10E63AEE31A0366F32651900012010DB
:10044000201020102010201020102010201000015B
:10045000201020102010201020102010201020101C
:10046000000120102010201020102010201020103B
:10047000201000012010201020102010201020102B
:10048000201020100000A01320088316870083127C
:100490002013200883168700831220122008831659
:1004A00087008312A0122008831687008512051288
:1004B00083122010200883168700831207108316EA
:1004C0000513831205171F139F1783169F17831297
:1004D0001F14831603170908C039890003131F125C
:1004E0009F120F30031788000030F80083120313A7
:1004F0001F08C33978049F008A150A164B284E300E
:100500008400831300080319922A0230F800F701CF
:10051000F70B882AF80B872A9730F700F70B8E2AFB
:10052000800B852A0800551E972A8717982A87135B
:10053000D51D9C2A05169D2A0512551DA12A851632
:10054000A22A8512D51CA62A8716A72A8712551C0F
:10055000AB2A0716AC2A071208000717AF2A0713A1
:10056000B12A08006430CE007F220330D5009322E8
:10057000AD220530CE007F220330D5009322AD227C
:100580000130CE007F220330D5009322AD2201300E
:10059000CE007F220230D5009322AD220130CE0062
:1005A0007F220230D5009322AD220130CE007F227F
:1005B0000E30D5009322AD220130CE007F22D5012E
:1005C0009322AD220130CE007F220830D500932245
:1005D000AD220130CE007F22D5019322AD22013021
:1005E000CE007F220C30D5009322AD220130CE0008
:1005F0007F22D5019322AD220130CE007F2206302A
:10060000D5009322AD220130CE007F22D501932266
:10061000AD220130CE007F220130D5009322AD22E1
:100620000230CE007F228A150A165B28D50193225C
:10063000AD220230D5009322AD220230CE007F22BF
:100640008A150A1660284E08003A0319312B013A20
:100650000319322B033A0319352B013A0319382BAE
:100660003B2B3C2B4030CD073C2B1430CD073C2B93
:100670005430CD073C2B3C2B80304D07D000500828
:10068000D100510EF7000F30F70577080F39D3006E
:1006900051080F39D2005308D5009322AD221A30E9
:1006A000F700F70B512B00005208D5009322AD2222
:1006B0001A30F700F70B5A2B00000800520ED30037
:1006C0000F30D305D20510305307D400D500932244
:1006D000AD2210305207D400D5009322AD221A303B
:1006E000F700F70B712B00000800831603178C1717
:1006F0000C140000000083120C087F390319B92B79
:100700000313CD0003170D080313CE0003170F08C2
:100710000313CF004D08D2005E234E0803178D004F
:1007200003134F0803178F0083168C170C14000057
:10073000000083120C0D0E0D7F390319B92B031322
:10074000CD0003170D080313CE0003170F08031382
:10075000CF004D08D2005E234E0803178D0003130F
:100760004F0803178F008D0A03198F0A0313752B87
:100770000317031308002015200883168700C02BD9
:10078000C12B83128710A010200883168700C82B66
:10079000C92B831207112011200883168700D02B44
:1007A000D12B83120800A014200883168700D82BB1
:1007B000D92B83122015200883168700DF2BE02B0E
:1007C000831207112011200883168700E72BE82BDE
:1007D000831208008710A010200883168700F02BD2
:1007E000F12B83122015200883168700F72BF82B96
:1007F000831207112011200883168700FF2B002C7D
:1008000083120800CC01A014200883168700082C4E
:10081000092C831220152008831687000F2C102C1A
:100820008312871C1B2C142C152CCC0A4C08643CFE
:1008300003191B2C112C0711201120088316870087
:10084000212C222C232C242C83128710A01020086A
:10085000831687002B2C2C2C83124C08643C031D20
:10086000462CCD01CE012323043003178D00003028
:100870008F00031375230430CD00FA30CE007F22A1
:10088000CD0B3D2C0130F800492C492C0030F800EC
:10089000492C08008710A010200883168700502CD0
:1008A000512C83122015200883168700572C582CB2
:1008B0008312A0142008831687005E2C5F2C8312FD
:1008C0000800BB23D323EA23EA23D323EA23D32339
:1008D000EA23EA230224F8080319722C4A2401307F
:1008E000F800A12CCB014B08073C031C802CC91F2E
:1008F0007B2CD3237C2CEA230310C90DCB0A732C49
:100900000224F8080319882C4A240130F800A12C8D
:10091000CB014B08073C031C962CCA1F912CD323F8
:10092000922CEA230310CA0DCB0A892C0224F80862
:1009300003199E2C4A240130F800A12C4A240030CF
:10094000F8000800BB23D323EA23EA23D323EA23B6
:10095000D323D323EA230224F8080319B32C4A240F
:100960000130F800E22CC6014608073C031CC12CEC
:10097000C41FBC2CD323BD2CEA230310C40DC60A0C
:10098000B42C0224F8080319C92C4A240130F800B9
:10099000E22CC6014608073C031CD72CC51FD22CED
:1009A000D323D32CEA230310C50DC60ACA2C022474
:1009B000F8080319DF2C4A240130F800E22C4A24FD
:1009C0000030F8000800BB23D323EA23EA23D32313
:1009D000EA23D323EA23EA230224F8080319F42C98
:1009E0004A240130F800812DCA014A08073C031C43
:1009F000022DC91FFD2CD323FE2CEA230310C90DA1
:100A0000CA0AF52C2015200883168700072D082D0B
:100A10008312A0142008831687000E2D0F2D831239
:100A200007112011200883168700162D172D831219
:100A300020152008831687001D2D1E2D8312871078
:100A4000A010200883168700252D262D831207115C
:100A500020112008831687002D2D2E2D8312D323DD
:100A6000EA23EA23D323EA23D323EA23D32302244A
:100A7000F80803193F2D4A240130F800812DCB01DD
:100A8000CA014A08073C031C682D0310CB0DA014B3
:100A900020088316870083122015200883168700FC
:100AA000512D522D8312871C582D0130CC00592D09
:100AB000CC01071120112008831687005F2D602DBF
:100AC00083124C08F800F808031D4B14CA0A412D84
:100AD000A0142008831687006D2D6E2D831220151B
:100AE000200883168700742D752D8312071120119D
:100AF0002008831687007C2D7D2D83124A244B0805
:100B0000F800080003178D0183168C130C14831250
:100B10000C08553C031DD72D03130618912D031700
:100B2000D72D0130C4004408093C031CA82D4408FB
:100B300003178D0083168C130C1483120C080313F7
:100B4000C5004408C9004508CA006124C40A932DA1
:100B5000553003178D0083168C130C1483120C0868
:100B60000313C5005530C9004508CA00612456303A
:100B700003178D0083168C130C1483120C080313B7
:100B8000C5005630C9004508CA0061245A30031711
:100B90008D0083168C130C1483120C080313C500EC
:100BA0005A30C9004508CA006124822E031701305B
:100BB0000313C4004408093C031C022E4408C90066
:100BC000E3247808C500440803178D000313450883
:100BD00003178C0083168C130C15831203130B0858
:100BE000F7008B138316031755308D00AA308D0044
:100BF0008C148C18F92D0C117708831203138B04B5
:100C0000C40ADA2D5530C900E3247808C5005530F0
:100C100003178D000313450803178C0083168C13EC
:100C20000C15831203130B08F7008B13831603179D
:100C300055308D00AA308D008C148C181D2E0C118F
:100C40007708831203138B045630C900E324780815
:100C5000C500563003178D000313450803178C0099
:100C600083168C130C15831203130B08F7008B13D8
:100C70008316031755308D00AA308D008C148C1804
:100C80003F2E0C117708831203138B045A30C900CE
:100C9000E3247808C5005A3003178D000313450874
:100CA00003178C0083168C130C15831203130B0887
:100CB000F7008B138316031755308D00AA308D0073
:100CC0008C148C18612E0C117708831203138B047B
:100CD00003178D0155308C0083168C130C1583126D
:100CE00003130B08F7008B138316031755308D0081
:100CF000AA308D008C148C187B2E0C11770883126F
:100D000003138B048A150A16BF285308F8015202F0
:100D100003188D2E5208F700992EF7010830D400E1
:100D2000D20DF70D530877020318F700F80DD40B16
:100D3000902E080020304D1E3030CE004C08F700B9
:100D4000CC1FA92EF709F70A7708CC002D30CE006A
:100D5000CD174C08D2006430D30085267708CC002C
:100D600030307807CF004C08D2000A30D3008526F7
:100D700030307707D10030307807D0004E08F700C8
:100D8000CD1DC42ECD1F4D114D1AD12ECD1FEC2ED1
:100D90004D19EC2E7708CF00CD18EC2E7708D00037
:100DA000EC2E30304F02031DEC2E7708CF002030A0
:100DB000CE00CD1DDF2E4D11CD14CD1FCD10303006
:100DC0005002031DEC2E7708D0002030CF00CD1D3F
:100DD000DF2ECD10CD1F4D104D1DF12E4E08D2002F
:100DE0005E23CD1CF62E4F08D2005E234D1CFB2E39
:100DF0005008D2005E235108D2005E230800303034
:100E00004902CA000310CA0C4908303CCB00031049
:100E1000CB0C490F132F093003178D0000308F00C2
:100E200003137523702F4908F73C0318232F2D3027
:100E3000D2005E234A08CC001330CD009A262E3013
:100E4000D2005E23702F4908433C0318362F203010
:100E5000D2005E232D30D2005E234A08CC00113030
:100E6000CD009A262E30D2005E23702F4908303CE8
:100E700003184C2F2030D2005E232030D2005E2396
:100E80002D30D2005E234A08CC001830CD009A26BF
:100E90002E30D2005E23702F49081C3C0318622FAD
:100EA0002030D2005E232030D2005E232030D200DA
:100EB0005E234B08CC001830CD009A262E30D2008D
:100EC0005E23702F2030D2005E232030D2005E23BC
:100ED0004B08CC001130CD009A262E30D2005E2374
:100EE000490F732F882F491C7F2F3530D2005E2386
:100EF0006430D2005E234230D2005E23882F30302F
:100F0000D2005E236430D2005E234230D2005E23E2
:100F10000800A1080319992FA2010618A20AA3012B
:100F20008618A30AA4010619A40AA5018619A50A10
:100F3000A101CA01C9010618C90A490822020319F8
:100F4000AB2F4908A2000A30CE007F22C908031D3A
:100F5000AB2F0130CA00C9018618C90A490823020B
:100F60000319BC2F4908A3000A30CE007F22C9080C
:100F7000031DBC2F0230CA00C9010619C90A49085D
:100F800024020319CD2F4908A4000A30CE007F2285
:100F9000C908031DCD2F0330CA00C9018619C90A2B
:100FA000490825020319DE2F4908A5000A30CE00A2
:100FB0007F22C908031DDE2F0430CA004A08F8004A
:020FC000080027
:101000004808003A03193228013A03193C28033AE8
:1010100003194628013A03195028073A03195A2898
:10102000013A03196428033A03196E28013A031997
:1010300078280F3A03198228013A03198C28033AB9
:1010400003199628013A0319A028073A0319AA2878
:10105000013A0319B428033A0319BE28013A0319C7
:10106000C828D2280D3003178D0000308F008A1158
:10107000031375238A15D328103003178D00003011
:101080008F008A11031375238A15D3281330031791
:101090008D0000308F008A11031375238A15D32821
:1010A000163003178D0000308F008A11031375234B
:1010B0008A15D328193003178D0000308F008A114C
:1010C000031375238A15D3281C3003178D000030B5
:1010D0008F008A11031375238A15D3281F30031735
:1010E0008D0000308F008A11031375238A15D328D1
:1010F000223003178D0000308F008A1103137523EF
:101100008A15D328253003178D0000308F008A11EF
:10111000031375238A15D328283003178D00003058
:101120008F008A11031375238A15D3282B300317D8
:101130008D0000308F008A11031375238A15D32880
:101140002E3003178D0000308F008A110313752392
:101150008A15D328313003178D0000308F008A1193
:10116000031375238A15D328343003178D000030FC
:101170008F008A11031375238A15D328373003177C
:101180008D0000308F008A11031375238A15D32830
:101190003A3003178D0000308F008A110313752336
:1011A0008A15D328D32808000230C9008A11E32405
:1011B0008A15F81FE5285A3003178D0001308F007B
:1011C0008A11031375238A15EE285E3003178D00EC
:1011D00001308F008A11031375238A155730C90017
:1011E0008A11E3248A157808C500C9008A11FF26F0
:1011F0008A15CD010130CE008A1123238A150730CC
:10120000C9008A11E3248A1578080139031D1229BF
:101210003D3003178D0000308F008A1103137523B2
:101220008A1546290830C9008A11E3248A157808EE
:10123000C500CD010130CE008A1123238A15543018
:10124000D2008A115E238A155230D2008A115E23A1
:101250008A15450EF7000F30F70577080F39C600DD
:10126000C80000202030D2008A115E238A15423047
:10127000D2008A115E238A155330D2008A115E2370
:101280008A1545080F39C600C80000208A11892731
:101290008A157808C4004408023C031D5229013015
:1012A000F8005929440B57290230F8005929003019
:1012B000F8008A150A165529831603178C170C1483
:1012C0000000000003188D2983120C087F390313D6
:1012D000CA0003170D080313CB0003170F080313ED
:1012E000CC004A08D2008A115E238A154B080317E6
:1012F0008D0003134C0803178F0083168C170C14F2
:101300000000000083120313C90B87298A29831662
:1013100003178D29AE298316031783120C0D0E0DAA
:101320007F390313CA0003170D080313CB000317FB
:101330000F080313CC004A08D2008A115E238A15D5
:101340004B0803178D0003134C0803178F008D0AF9
:1013500003198F0A03100313C90B5C2908004D30D1
:10136000D2008A115E238A154408CC001F30CD00BC
:101370008A119A268A15463003178D0000308F0097
:1013800003140E300313C9005C21CD010130CE00DF
:101390008A1123238A154E3003178D0000308F00E9
:1013A0008A11031375238A150830C9008A11E324B2
:1013B0008A157808C600460EF7000F30F705770843
:1013C0000F39C6004608C80000206430D2008A11D8
:1013D0005E238A154230D2008A115E238A154608A0
:1013E000C5008A1189278A157808C7004708033C79
:1013F000031D012AC60A4608103C031D012A0F30AE
:10140000C6004708043C031D082AC608031DC6037E
:10141000460845020319422A0830C9008A11E3240C
:101420008A157808C5000F30C505460EF700F03064
:10143000F7057708F039C6004608C5040830C9002A
:101440004508CA008A1161248A15083003178D00E7
:101450000313450803178C0083168C130C15831295
:1014600003130B08F7008B138316031755308D00F9
:10147000AA308D008C148C183B2A0C11770883122B
:1014800003138B04470B472A0230F800502A470801
:10149000023C031D4E2A0130F800502A0030F800AB
:1014A0008A150A165D294D30D2008A115E238A15ED
:1014B0004408CC001F30CD008A119A268A1552307C
:1014C00003178D0000308F0003140E300313C90082
:1014D0005C21CD010130CE008A1123238A155A30B8
:1014E00003178D0000308F008A11031375238A15AE
:1014F0000830C9008A11E3248A157808C6000F3025
:10150000C6054608C80000206430D2008A115E2358
:101510008A154230D2008A115E238A154608C5001A
:101520008A1189278A157808C7004708033C031DDC
:10153000A02AC60A4608103C031DA02A0F30C60088
:101540004708043C031DA72AC608031DC603460816
:1015500045020319DA2A0830C9008A11E3248A15E2
:101560007808C500F030C5054608C5040830C90034
:101570004508CA008A1161248A15083003178D00B6
:101580000313450803178C0083168C130C15831264
:1015900003130B08F7008B138316031755308D00C8
:1015A000AA308D008C148C18D32A0C117708831262
:1015B00003138B04470BDF2A0230F800E82A4708A0
:1015C000023C031DE62A0130F800E82A0030F8004A
:1015D0008A150A1665294D30D2008A115E238A15B4
:1015E0004408CC001F30CD008A119A268A155E303F
:1015F00003178D0000308F0003140E300313C90051
:101600005C21CD010130CE008A1123238A1566307A
:1016100003178D0000308F008A11031375238A157C
:101620000730C9008A11E3248A157808C500C6006E
:10163000C7001830C60546080319282B083A0319B5
:10164000322B183A03193C2B083A0319462B502B1E
:101650006A3003178D0000308F008A110313752341
:101660008A15512B6D3003178D0000308F008A11C1
:10167000031375238A15512B703003178D0000302A
:101680008F008A11031375238A15512B73300317AA
:101690008D0000308F008A11031375238A15512B9A
:1016A000512B8A1189278A157808C8004808043CFC
:1016B000031D5E2B0830C6071830C6054808033CDA
:1016C000031D662B0830C6021830C605E730C50575
:1016D0004608C504470845020319922B0730C90084
:1016E0004508CA008A1161248A15073003178D0046
:1016F0000313450803178C0083168C130C158312F3
:1017000003130B08F7008B138316031755308D0056
:10171000AA308D008C148C188B2B0C117708831237
:1017200003138B04480B972B0230F800A02B4808BA
:10173000023C031D9E2B0130F800A02B0030F80066
:101740008A150A166D294D30D2008A115E238A153A
:101750004408CC001F30CD008A119A268A157730B4
:1017600003178D0000308F0003140C300313C900E1
:101770005C21CD010130CE008A1123238A157E30F1
:1017800003178D0000308F008A11031375238A150B
:101790000730C9008A11E3248A157808C500C600FD
:1017A000C7000630C60546080319E02B023A0319A4
:1017B000EA2B063A0319F42B023A0319FE2B082CE4
:1017C000823003178D0000308F008A1103137523B8
:1017D0008A15092C863003178D0000308F008A117E
:1017E000031375238A15092C8A3003178D000030E6
:1017F0008F008A11031375238A15092C8E30031765
:101800008D0000308F008A11031375238A15092C6F
:10181000092C8A1189278A157808C8004808043CD1
:10182000031D162C0230C6070630C6054808033CC7
:10183000031D1E2C0230C6020630C605F930C50550
:101840004608C5044708450203194A2C0730C90059
:101850004508CA008A1161248A15073003178D00D4
:101860000313450803178C0083168C130C15831281
:1018700003130B08F7008B138316031755308D00E5
:10188000AA308D008C148C18432C0C11770883120D
:1018900003138B04480B4F2C0230F800582C4808D7
:1018A000023C031D562C0130F800582C0030F80083
:1018B0008A150A1675294D30D2008A115E238A15C1
:1018C0004408CC001F30CD008A119A268A15933027
:1018D00003178D0000308F0003140C300313C90070
:1018E0005C21CD010130CE008A1123238A152030DE
:1018F000D2008A115E238A150930C9008A11E324B7
:101900008A157808C500C600C7003830C6054608E5
:101910000319A02C083A0319AA2C183A0319B42C5D
:10192000083A0319BE2C383A0319C82C083A03198F
:10193000D22C183A0319DC2C083A0319E62CF02CA7
:101940009A3003178D0000308F008A11031375231E
:101950008A15F12CA03003178D0000308F008A11FA
:10196000031375238A15F12CA63003178D00003060
:101970008F008A11031375238A15F12CAC300317DD
:101980008D0000308F008A11031375238A15F12C06
:10199000B23003178D0000308F008A1103137523B6
:1019A0008A15F12CB83003178D0000308F008A1192
:1019B000031375238A15F12CBE3003178D000030F8
:1019C0008F008A11031375238A15F12CC430031775
:1019D0008D0000308F008A11031375238A15F12CB6
:1019E000F12C8A1189278A157808C8004808043C18
:1019F000031DFE2C0830C6073830C6054808033CD6
:101A0000031D062D0830C6023830C605C730C5058F
:101A10004608C504470845020319322D0930C9009C
:101A20004508CA008A1161248A15093003178D0000
:101A30000313450803178C0083168C130C158312AF
:101A400003130B08F7008B138316031755308D0013
:101A5000AA308D008C148C182B2D0C117708831252
:101A600003138B04480B372D0230F800402D480833
:101A7000023C031D3E2D0130F800402D0030F800DF
:101A80008A150A167D294D30D2008A115E238A15E7
:101A90004408CC001F30CD008A119A268A15FB30ED
:101AA00003178D0000308F0003140C300313C9009E
:101AB0005C21CD010130CE008A1123238A1520300C
:101AC000D2008A115E238A155530C9008A11E32499
:101AD0008A157808C500C600C7000830C605460844
:101AE0000319762D083A0319802D8A2D0230031729
:101AF0008D0001308F008A11031375238A158B2DF9
:101B0000083003178D0001308F008A1103137523ED
:101B10008A158B2D8B2D8A1189278A157808C80084
:101B20004808043C031D972D0830C607C605480821
:101B3000033C031D9E2D0830C602C605C51146088C
:101B4000C504470845020319C92D5530C900450889
:101B5000CA008A1161248A15553003178D000313BA
:101B6000450803178C0083168C130C15831203137E
:101B70000B08F7008B138316031755308D00AA301E
:101B80008D008C148C18C22D0C117708831203134E
:101B90008B04480BCE2D0230F800D72D4808023CAC
:101BA000031DD52D0130F800D72D0030F8008A151F
:101BB0000A1685294D30D2008A115E238A15440801
:101BC000CC001F30CD008A119A268A150F300317DA
:101BD0008D0001308F0003140C300313C9005C2109
:101BE000CD010130CE008A1123238A151630031748
:101BF0008D0001308F008A11031375238A1555302B
:101C0000C9008A11E3248A157808C500C600C700F8
:101C10000730C60546080319232E013A03192D2E55
:101C2000033A0319372E013A0319412E073A0319D3
:101C30004B2E013A0319552E033A03195F2E013A30
:101C40000319692E732E193003178D0001308F0090
:101C50008A11031375238A15742E1E3003178D0005
:101C600001308F008A11031375238A15742E2330D7
:101C700003178D0001308F008A11031375238A1515
:101C8000742E283003178D0001308F008A11031342
:101C900075238A15742E2D3003178D0001308F00A7
:101CA0008A11031375238A15742E323003178D00A1
:101CB00001308F008A11031375238A15742E373073
:101CC00003178D0001308F008A11031375238A15C5
:101CD000742E3C3003178D0001308F008A110313DE
:101CE00075238A15742E742E8A1189278A1578080F
:101CF000C8004808043C031D812E0130C607073088
:101D0000C6054808033C031D892E0130C602073072
:101D1000C605F830C5054608C5044708450203193D
:101D2000B52E5530C9004508CA008A1161248A15AC
:101D3000553003178D000313450803178C008316D5
:101D40008C130C15831203130B08F7008B138316E7
:101D5000031755308D00AA308D008C148C18AE2ED0
:101D60000C117708831203138B04480BBA2E023030
:101D7000F800C32E4808023C031DC12E0130F800B4
:101D8000C32E0030F8008A150A168D294A08003A39
:101D90000319F82E013A0319022F033A03190C2FE5
:101DA000013A0319162F073A0319202F013A031994
:101DB0002A2F033A0319342F013A03193E2F0F3A01
:101DC0000319482F013A0319522F033A03195C2FC4
:101DD000013A0319662F073A0319702F013A0319C4
:101DE0007A2F033A0319842F013A03198E2F982F63
:101DF000CA3003178D0000308F008A11031375233A
:101E00008A15992FCD3003178D0000308F008A116D
:101E1000031375238A15992FD03003178D000030D6
:101E20008F008A11031375238A15992FD330031756
:101E30008D0000308F008A11031375238A15992FA6
:101E4000D63003178D0000308F008A1103137523DD
:101E50008A15992FD93003178D0000308F008A1111
:101E6000031375238A15992FDC3003178D0000307A
:101E70008F008A11031375238A15992FDF300317FA
:101E80008D0000308F008A11031375238A15992F56
:101E9000E23003178D0000308F008A110313752381
:101EA0008A15992FE53003178D0000308F008A11B5
:101EB000031375238A15992FE83003178D0000301E
:101EC0008F008A11031375238A15992FEB3003179E
:101ED0008D0000308F008A11031375238A15992F06
:101EE000EE3003178D0000308F008A110313752325
:101EF0008A15992FF13003178D0000308F008A1159
:101F0000031375238A15992FF43003178D000030C1
:101F10008F008A11031375238A15992FF730031741
:101F20008D0000308F008A11031375238A15992FB5
:101F3000992F6430D2008A115E238A154230D20074
:101F40008A115E238A1508004D0DF700F70DFC304D
:101F5000F7051F08C33977049F001A30F700F70B05
:101F6000AF2F0000CF01CE01D00150080F3C031C61
:101F7000D92F9F1451109F1C51145118C32F511069
:101F80009F1C5114BD2F9F18C32F1E08FA008316E3
:101F90001E088312D2001E08D3005208F80053080E
:101FA000F9007808CE0779080318790FCF07D00A0F
:101FB000B52FCF0CCE0CCF0CCE0CCF0CCE0CCF0C43
:101FC000CE0C0F30CF054E08F8004F08F90008007E
:102000004D30D2000A125E230A164408CC001F305D
:10201000CD000A129A260A16423003178D000130AD
:102020008F0003140D300313C9000A128A155C21B6
:102030000A168A11CD010130CE000A1223230A1696
:102040004A3003178D0001308F000A1203137523E5
:102050000A165630C9000A12E3240A167808C50089
:10206000C600C700460EF7000F30F70577080F3996
:10207000C900CA000A128A15C6260A168A110A124F
:1020800089270A167808C8004808043C031D4C2814
:102090001030C607F030C6054808033C031D54281D
:1020A0001030C602F030C6050F30C5054608C5041D
:1020B00047084502031980285630C9004508CA0060
:1020C0000A1261240A16563003178D0003134508BF
:1020D00003178C0083168C130C15831203130B0843
:1020E000F7008B138316031755308D00AA308D002F
:1020F0008C148C1879280C117708831203138B0425
:10210000480B85280230F8008E284808023C031D41
:102110008C280130F8008E280030F8008A150A1645
:1021200095294D30D2000A125E230A164408CC00CD
:102130001F30CD000A129A260A164F3003178D0061
:1021400001308F0003140E300313C9000A128A15E0
:102150005C210A168A11CD010130CE000A12232318
:102160000A16573003178D0001308F000A1203132F
:1021700075230A165630C9000A12E3240A16780895
:10218000C500C600C70046080F39C900CA000A12B8
:102190008A15C6260A168A110A1289270A1678088D
:1021A000C8004808043C031DD9280130C6070F3079
:1021B000C6054808033C031DE1280130C6020F3064
:1021C000C605F030C5054608C50447084502031991
:1021D0000D295630C9004508CA000A1261240A16A2
:1021E000563003178D000313450803178C00831620
:1021F0008C130C15831203130B08F7008B13831633
:10220000031755308D00AA308D008C148C180629C8
:102210000C117708831203138B04480B1229023028
:10222000F8001B294808023C031D19290130F80059
:102230001B290030F8008A150A169D294D30D2005E
:102240000A125E230A164408CC001F30CD000A1281
:102250009A260A16633003178D0001308F0003148D
:102260000C300313C9000A128A155C210A168A1160
:10227000CD010130CE000A1223230A160430C90012
:102280000A12E3240A167808C500C600C7004708EA
:10229000C03903195229403A03195C29C03A03197D
:1022A000662970296A3003178D0001308F000A12E9
:1022B000031375230A167129733003178D0001303B
:1022C0008F000A12031375230A1671297C30031735
:1022D0008D0001308F000A12031375230A1671292D
:1022E00071290A1289270A167808C8004808043C90
:1022F000031D81294030C607C6054608C03C0319A6
:10230000C6014808033C031D8E294030C602C6059D
:102310004608C03C031D8E298030C6003F30C505ED
:102320004608C504470845020319CD295F30C90096
:10233000FF30CA000A1261240A160A30CE000A12BF
:102340007F220A160430C9004508CA000A12612417
:102350000A16043003178D000313450803178C0079
:1023600083168C130C15831203130B08F7008B13C1
:102370008316031755308D00AA308D008C148C18ED
:10238000BF290C117708831203138B045F30C90037
:10239000E030CA000A1261240A16480BD229023022
:1023A000F800DB294808023C031DD9290130F80058
:1023B000DB290030F8008A150A16A5294D30D20015
:1023C0000A125E230A164408CC001F30CD000A1200
:1023D0009A260A16863003178D0001308F000314E9
:1023E0000A300313C9000A128A155C210A168A11E1
:1023F000CD010130CE000A1223230A162030D2006C
:102400000A125E230A162030D2000A125E230A1630
:102410002030D2000A125E230A160630C9000A12C2
:10242000E3240A167808C500C600C70047080C391F
:102430000319242A043A03192E2A0C3A0319382ABC
:10244000043A0319422A4C2A8C3003178D000130BC
:102450008F000A12031375230A164D2A92300317B0
:102460008D0001308F000A12031375230A164D2ABE
:10247000983003178D0001308F000A120313752363
:102480000A164D2A9E3003178D0001308F000A1264
:10249000031375230A164D2A4D2A0A1289270A1694
:1024A0007808C8004808043C031D5A2A0430C607AF
:1024B0000C30C6054808033C031D622A0430C602DE
:1024C0000C30C605F330C5054608C504470845026B
:1024D00003198E2A0630C9004508CA000A12612471
:1024E0000A16063003178D000313450803178C00E6
:1024F00083168C130C15831203130B08F7008B1330
:102500008316031755308D00AA308D008C148C185B
:10251000872A0C117708831203138B04480B932A24
:102520000230F8009C2A4808023C031D9A2A013018
:10253000F8009C2A0030F8008A150A16AD294D30A3
:10254000D2000A125E230A164408CC001F30CD00C8
:102550000A129A260A16A53003178D0001308F0043
:1025600003140A300313C9000A128A155C210A16E3
:102570008A11CD010130CE000A1223230A16203021
:10258000D2000A125E230A162030D2000A125E23FD
:102590000A162030D2000A125E230A160630C9003D
:1025A0000A12E3240A167808C500C600C7004708C7
:1025B00003390319E52A013A0319EF2A033A0319EB
:1025C000F92A013A0319032B0D2BAB3003178D00A9
:1025D00001308F000A12031375230A160E2BB13037
:1025E00003178D0001308F000A12031375230A169A
:1025F0000E2BB73003178D0001308F000A12031322
:1026000075230A160E2BBD3003178D0001308F0085
:102610000A12031375230A160E2B0E2B0A12892792
:102620000A167808C8004808043C031D1B2B01301B
:10263000C6070330C6054808033C031D232B0130A1
:10264000C6020330C605FC30C5054608C504470868
:10265000450203194F2B0630C9004508CA000A126B
:1026600061240A16063003178D000313450803176B
:102670008C0083168C130C15831203130B08F700C0
:102680008B138316031755308D00AA308D008C14E0
:102690008C18482B0C117708831203138B04480BFA
:1026A000542B0230F8005D2B4808023C031D5B2BC5
:1026B0000130F8005D2B0030F8008A150A16B529A4
:1026C0004D30D2000A125E230A164408CC001F3097
:1026D000CD000A129A260A16C43003178D00013065
:1026E0008F0003140B300313C9000A128A155C21F2
:1026F0000A168A11CD010130CE000A1223230A16D0
:10270000CB3003178D0001308F000A12031375239D
:102710000A165A30C9000A12E3240A167808C500BE
:10272000C600C7004708C9000A12FF260A160A1287
:1027300089270A167808C8004808033C031DA82BFF
:102740000130C6074608573C0318A82B5830C6006E
:102750004808043C031DB42B0130C6024608083C5F
:10276000031CB42B0830C6004608C50047084502C4
:102770000319DE2B5A30C9004508CA000A12612429
:102780000A165A3003178D000313450803178C00EF
:1027900083168C130C15831203130B08F7008B138D
:1027A0008316031755308D00AA308D008C148C18B9
:1027B000D72B0C117708831203138B04480BE32BE0
:1027C0000230F800EC2B4808023C031DEA2B0130D4
:1027D000F800EC2B0030F8008A150A16BD294D30A0
:1027E000D2000A125E230A164408CC001F30CD0026
:1027F0000A129A260A16D03003178D0001308F0076
:1028000003140B300313C9000A128A155C210A163F
:102810008A11CD010130CE000A1223230A1602309C
:10282000C9000A12E3240A167808C500C600C700CA
:102830004708073903192C2C013A0319362C033A9F
:102840000319402C013A03194A2C073A0319542C56
:10285000013A03195E2C682CD73003178D00013024
:102860008F000A12031375230A16692CE030031730
:102870008D0001308F000A12031375230A16692C8C
:10288000E93003178D0001308F000A1203137523FE
:102890000A16692CF23003178D0001308F000A12DE
:1028A000031375230A16692CFB3003178D000130C2
:1028B0008F000A12031375230A16692C04300317BC
:1028C0008D0002308F000A12031375230A16692C3B
:1028D000692C0A1289270A167808C8004808043C9F
:1028E000031D7A2C0130C6070730C6054608063C92
:1028F0000319C6014808033C031D882C0130C60299
:102900000730C6054608073C031D882C0530C60065
:10291000F830C5054608C504470845020319B42C1C
:102920000230C9004508CA000A1261240A160230A2
:1029300003178D000313450803178C0083168C13AF
:102940000C15831203130B08F7008B138316031760
:1029500055308D00AA308D008C148C18AD2C0C11C4
:102960007708831203138B04480BB92C0230F8004C
:10297000C22C4808023C031DC02C0130F800C22CB8
:102980000030F8008A150A16C529F801F901F70187
:10299000FA014C08031DCF2C4B080319E92C103009
:1029A000CD000310C90DCA0DF70DFA0D4C087A02BF
:1029B000031DDC2C4B087702031CE52C4B08F702A7
:1029C000031CFA034C08FA020314F80DF90DCD0BA1
:1029D000D12C0800C701B3080319182DCA014A08F1
:1029E000033C031C172D03104A0D343EF800FA0176
:1029F0000318FA0A7808CB007A08CC004708CD0003
:102A00000A128A15A4270A168A114B088400831318
:102A10004C188317840A79088000840378088000A2
:102A20003C304A07840083138001CA0AEF2CB301AB
:102A30004708CD000A128A15A4270A168A117908B8
:102A4000C9007808C8003C30470784008313000B96
:102A5000772D0310470D343E84008313840A000849
:102A6000CC0084030008CB004C084902031C4A2D0B
:102A7000031D3E2D48084B0203184A2D0310470D35
:102A8000343E84008313840A490880008403480884
:102A90008000762D0310470D343E84008313840A92
:102AA0000008CC0084030008CB0001304807F80080
:102AB0004908FA000318FA0A7A084C02031C762D1A
:102AC000031D662D4B0878020318762D0310470D61
:102AD000343E84008313840A490880008403480834
:102AE00080003C304707840083138001C22D03100F
:102AF000470D343E84008313840A0008CC0084030D
:102B00000008CB0049084C02031C982D031D8C2D96
:102B10004B0848020318982D0310470D343E8400DB
:102B20008313840A49088000840348088000C22D6A
:102B30000310470D343E84008313840A0008CC0040
:102B400084030008CB000130CB070318CC0A4C08E3
:102B50004902031CC22D031DB12D48084B02031866
:102B6000C22D0310470D343E84008313840A4908A4
:102B700080008403480880003C30470784008313AA
:102B8000013080000310470D343E84008313000899
:102B9000F800840A00088403F9007908C500780861
:102BA000C4004508013C031CE72D0310C40DC50DEE
:102BB0004508CA004408C900CC010730CB00C52431
:102BC0007908C5007808C400FF3CC600FB2D003022
:102BD0004402C7004508C8000230031C0330C80285
:102BE0004808CA004708C900CC010730CB00C524FB
:102BF00078086D3CC600460840020319082E57307D
:102C0000C9004608CA000A1261240A164608C00014
:102C10008A150A160A2A0230C9000A12E3240A1683
:102C20007808C400061B1F2EC41F1E2EC4130230BA
:102C3000C9004408CA000A1261240A162B2E44084F
:102C40008039031D2B2EC4170230C9004408CA0066
:102C50000A1261240A168A150A160D2A0730C900BD
:102C60000A12E3240A167808C400861A442E44087F
:102C70000139031D432E44140730C9004408CA001B
:102C80000A1261240A164E2E441C4E2E44100730A0
:102C9000C9004408CA000A1261240A168A150A16D5
:022CA000102AF8
:10300000840183131F308305713083168F000F08EE
:10301000FF308312A0000130A1000130A600013072
:10302000B300FF30C0008830C100831603170908C1
:10303000C039890003131F129F1200300317880044
:1030400083128701880189010313A201A301A4014E
:10305000A501A701A801A901AA01AB01AC01AD011D
:10306000AE01AF01B001B101B201B401B501B601C9
:10307000B701B801B901BA01BB01BC01BD01BE0174
:10308000BF01FF30831685008600870089150A126C
:103090008A118312432A0A168A150230C400FA30B4
:1030A000CE000A128A117F220A168A15C40B4F28F5
:1030B0000A128A11B22A0A168A150A128A11162BC6
:1030C0000A168A15CD01CE010A128A1123230A1687
:1030D0008A150D3003178D0002308F000A128A11F5
:1030E000031375230A168A150230C400FA30CE0085
:1030F0000A128A117F220A168A15C40B7628071431
:103100006430CE000A128A117F220A168A15FF3017
:103110008316950081138312CD010130CE000A126F
:103120008A1123230A168A15163003178D000230E0
:103130008F000A128A11031375230A168A150230AA
:10314000C400FA30CE000A128A117F220A168A15AC
:10315000C40BA1285730C900FF30CA000A128A11D7
:1031600061240A168A155730C400FF30C5000A12C0
:103170008A11A2240A168A150A128A11822D0A16A9
:103180008A155530C9000A128A11E3240A168A15D5
:103190007808C300C3155530C9004308CA000A1295
:1031A0008A1161240A168A155F30C900E030CA000E
:1031B0000A128A1161240A168A155F30C400E030B1
:1031C000C5000A128A11A2240A168A15C201033008
:1031D000C9008F30CA000A128A1161240A168A15A2
:1031E0005730C4003030C5000A128A11A2240A16D2
:1031F0008A15CD01CE010A128A1123230A168A15D7
:103200001F3003178D0002308F000A128A1103133A
:1032100075230A168A15CD010130CE000A128A11D3
:1032200023230A168A15283003178D0002308F00D9
:103230000A128A11031375230A168A15CD01CE01CD
:103240000A128A1123230A168A15420803195329E0
:10325000013A03195929033A03196129013A03195B
:103260006929073A03197129013A03197929033A9F
:1032700003198129013A031989290F3A0319912960
:10328000013A03199929033A0319A129013A0319AB
:10329000A929073A0319B129013A0319B929033AAF
:1032A0000319C129C9290A12D4280A167808C300AB
:1032B000CA294208C4000A12AF290A167808C300B6
:1032C000CA294208C4000A12532A0A167808C30001
:1032D000CA294208C4000A12EB2A0A167808C30059
:1032E000CA294208C4000A12A32B0A167808C30090
:1032F000CA294208C4000A125B2C0A167808C300C7
:10330000CA294208C4000A12432D0A167808C300CD
:10331000CA294208C4000A12DA2D0A167808C30026
:10332000CA294208C4008A1100288A157808C300F7
:10333000CA294208C4008A1191288A157808C30056
:10334000CA294208C4008A111E298A157808C300B8
:10335000CA294208C4008A11DE298A157808C300E8
:10336000CA294208C4008A119F2A8A157808C30016
:10337000CA294208C4008A11602B8A157808C30044
:10338000CA294208C4008A11EF2B8A157808C300A5
:10339000CA29CA29430BCD29D1294308023C031D60
:1033A000F629CD01CE010A128A1123230A168A15A5
:1033B000313003178D0002308F000A128A11031377
:1033C00075230A168A15CD010130CE000A128A1122
:1033D00023230A168A153A3003178D0002308F0016
:1033E0000A128A11031375230A168A15430BF92949
:1033F000C20A42080F3C0319C2014308023C031DE4
:10340000082AC208031D072A0E30C200082AC20378
:103410008A11EA2C8A158A110B2E8A158A112E2EF2
:063420008A151E2963005D
:04400E00842FFF3FBD
:00000001FF
